:100000000C9422010C943F010C943F010C943F018D
:100010000C943F010C943F010C943F010C943F0160
:100020000C943F010C943F010C943F010C943F0150
:100030000C943F010C943F010C943F010C943F0140
:100040000C943F010C943F010C943F010C943F0130
:100050000C943F010C943F010C943F010C943F0120
:100060000C943F010C943F01000000000000065F6B
:1000700006000703000703247E247E24242B6A1233
:1000800000631308646336495620500007030000DC
:10009000003E41000000413E0000083E1C3E0808B2
:1000A000083E080800E06000000808080808006032
:1000B00060000020100804023E5149453E00427F86
:1000C0004000625149494622494949361814127F75
:1000D0001027454545393C4A494930017109050316
:1000E0003649494936064949291E006C6C00000012
:1000F000EC6C000008142241002424242424004134
:1001000022140802015909063E415D551E7E090967
:10011000097E7F494949363E414141227F41414163
:100120003E7F494949417F090909013E4149497AD0
:100130007F0808087F00417F4100304040403F7FFA
:10014000081422417F404040407F0204027F7F022A
:1001500004087F3E4141413E7F090909063E415165
:10016000215E7F09091966264949493201017F014B
:10017000013F4040403F1F2040201F3F403C403F48
:1001800063140814630708700807714945430000A9
:100190007F41410002040810200041417F00040219
:1001A00001020480808080800003070000205454F6
:1001B00054787F44444438384444442838444444C0
:1001C0007F3854545418087E09090018A4A4A47C4C
:1001D0007F0404780000007D00004080847D007F63
:1001E0001028440000007F40007C041804787C0440
:1001F0000478003844444438FC4444443838444487
:1002000044FC44784404080854545420043E4424D4
:10021000003C40207C001C2040201C3C6030603CA6
:100220006C10106C009CA0603C006454544C00089E
:100230003E41410000007F00000041413E080201B4
:100240000201000011241FBECFEFD8E0DEBFCDBFFA
:1002500012E0A0E0B1E0E4EEFCE102C005900D92F6
:10026000AC3AB107D9F716E0ACEAB2E001C01D9292
:10027000A03FB107E1F70E94F50B0C94700E0C94AF
:10028000000040EA5FE009C020E0FA013197F1F791
:100290002F5F2F3FD1F78F5F90408F3F910509F07F
:1002A00098F7009749F020E040EA5FE0FA013197C3
:1002B000F1F72F5F2817D0F308954F925F927F9246
:1002C0008F929F92AF92BF92CF92DF92EF92FF9266
:1002D0000F931F93CF93DF937B018C014A01290178
:1002E0002115310509F466C097FF0DC08DE2FA01B2
:1002F0008083AA24BB246501AE18BF08C00AD10AB6
:10030000C1E0D0E016C0611571058105910569F461
:10031000AA24BB24650141E0E42EF12C012D112D0E
:10032000C0E0D0E0772473943CC05B016C01C0E076
:10033000D0E0E12C3AECF32E3AE9032F3BE3132F04
:1003400077242FC0AE14BF04C006D10610F4772066
:10035000E1F0C601B501A80197010E943A0EF4012F
:10036000EC0FFD1F205D20832053219630E040E0FC
:1003700050E0CA01B901A80197010E94080EA61A0F
:10038000B70AC80AD90A77247394C801B7012AE0CA
:1003900030E040E050E00E943A0EC901DA017C01F1
:1003A0008D01C415D50530F4E114F10401051105E2
:1003B00049F611C0C401DF91CF911F910F91FF90B9
:1003C000EF90DF90CF90BF90AF909F908F907F90F5
:1003D0005F904F900895C80DD91D1882EBCF8F9272
:1003E0009F92AF92BF92CF92DF92EF92FF920F93C4
:1003F0001F93CF93DF935C016B01EA014901401722
:10040000510719F0A0E0B0E069C040E050E008C03A
:10041000F501E40FF51F8081882329F04F5F5F4FBE
:100420004C155D05A8F34E155F0518F0A0E0B0E08F
:1004300043C0A0E0B0E007C0FE01EA0FFB1F8081CF
:10044000882321F01196A815B905B0F3B701641BF4
:10045000750B6A177B0708F0BD01DE01A60FB71FF9
:10046000FB01E40FF51FEC0FFD1F9B0104C02150A1
:1004700030408C9180831197319721153105B9F760
:1004800006C0FE01E20FF31F80832F5F3F4F2C1544
:100490003D0548F42E153F0530F4F501E20FF31F3A
:1004A0008081882371F7D901A60FB71F43C0F801D7
:1004B000EA0FFB1F80831196AC15BD05D8F5AE156C
:1004C000BF05F0F5F501EA0FFB1F8081882379F75E
:1004D00034C0F801EA0FFB1F80831196AC15BD05EF
:1004E00050F4AE15BF0560F5F501EA0FFB1F8081E2
:1004F000882379F703C0AE15BF05E0F498012A0FF1
:100500003B1FA7014A1B5B0B80E090E005C0F9018F
:10051000E80FF91F608301968815990548F4841740
:10052000950730F4FE01E80FF91F6081662379F723
:10053000A80FB91FAE15BF0518F4A00FB11F1C926C
:10054000DF91CF911F910F91FF90EF90DF90CF90AF
:10055000BF90AF909F908F900895CF93DF93EC0161
:10056000A0E0B0E005C0FA01EA0FFB1F80831196FE
:10057000A617B70750F4A217B30768F4FE01EA0FF5
:10058000FB1F8081882379F703C0A217B30718F4F3
:10059000A40FB51F1C92DF91CF9108958093BB00EB
:1005A00088E290E00197F1F784E88093BC008091A5
:1005B000BC0087FFFCCF8091B900887F883191F023
:1005C0008091B900887F883269F08091B900887F76
:1005D000803441F08091B90090E0887F803519F037
:1005E00091E001C090E0892F0895549889B18071FD
:1005F00090E054E0959587955A95E1F7982F8111F1
:1006000091E0892F08958091CB029091CB028F3F8A
:1006100011F097FD04C08091CB028F3F19F4109226
:10062000CB023FC01092BE029091CB028091BE02DD
:10063000282F30E040E050E0933010F441E050E0EB
:1006400024233523232B69F1239A2B9A20E040EAB7
:100650005FE0CA010197F1F72F5F2A3FD1F720E051
:1006600040EA5FE0CA010197F1F72F5F2A3FD1F717
:1006700020E040EA5FE0CA010197F1F72F5F2A3FCF
:10068000D1F720E040EA5FE0CA010197F1F72F5F60
:100690002A3FD1F78091B50285EC8093B502239A69
:1006A0002B989091C5028091CB02981739F4109243
:1006B000B8021092C5021092CB020EC08091CB02FC
:1006C0008093C5029091B8028091CB02891720F0E7
:1006D0008091C5028093B8029091B8028091C402C3
:1006E000891740F5239A2B9A84EF91E00E944101EB
:1006F000239A2B9885EC8093B5028091C902909142
:10070000CA02069774F08091C1029091C2020196CC
:100710009093C2028093C1021092CA021092C90241
:1007200009C08091C9029091CA0201969093CA02B1
:100730008093C9029091AF028091B802981720F47B
:100740008091B8028093AF0208951F93182F84EA16
:100750008093BC008091BC0087FFFCCF8091B002E9
:100760000E94CE0280E00E94CE02812F0E94CE0223
:1007700084E98093BC001F910895CF92DF92EF929D
:10078000FF920F931F93DF93CF93CDB7DEB7699797
:100790000FB6F894DEBF0FBECDBF69E170E040E058
:1007A00051E020E030E06E010894C11CD11C8601AC
:1007B000E9E1EE2EF12C0E94EF0120E030E0A601ED
:1007C000FA01E20FF31F8081882329F02F5F3F4F4A
:1007D00029313105A9F7922FAE014F5F5F4FFA0122
:1007E00020E030E008C0220F331F8081813311F4F4
:1007F0002F5F3F4F31968E2F841B8917A1F7E0EAB8
:10080000FFE03197F1F7C90169960FB6F894DEBFA2
:100810000FBECDBFCF91DF911F910F91FF90EF9051
:10082000DF90CF9008959F92AF92BF92CF92DF92C8
:10083000EF92FF920F931F93DF93CF9300D000D0DE
:10084000CDB7DEB780910501909106019A83898327
:100850009C838B8381E091E062E070E0AE014F5FAA
:100860005F4F22E030E00E94AD0281E091E062E063
:1008700070E0AE014D5F5F4F22E030E00E94AD02BC
:1008800081E091E062E070E049E952E021E130E08E
:100890000E94AD02539A5B98549A5C9A1092C702D8
:1008A0001092C80211E006C00E94F502882311F4DC
:1008B0001093C7028091C7028823B1F31092C70238
:1008C0001092B2021092B102A8E2CA2ED12C5E019F
:1008D0000894A11CB11C992493948091C80288317A
:1008E00078F09092C702539A5B9A539A5B98539A06
:1008F0005B9A539A5B98539A5B9A539A5B984BC056
:100900008091C802803158F0539A5B9AC6010197D2
:10091000F1F7539A5B98C6010197F1F73CC08091BB
:10092000C802883088F0539A5B9AC6010197F1F7A4
:10093000539A5B98C6010197F1F789E992E061E16A
:1009400070E043E051E01FC0539A5B9AC6010197E3
:10095000F1F7539A5B98C6010197F1F7549860E05C
:1009600070E080E090E04C9B04C061E070E080E0CB
:1009700090E0A50122E030E00E945D0189E992E06B
:1009800061E170E0A50122E030E08C01F1E1EF2EA1
:10099000F12C0E94EF018091C8028F5F8093C80202
:1009A0008091C702882309F498CF89E992E00E94D8
:1009B000BD039093B2028093B1026091B102709135
:1009C000B202882777FD8095982F0E94190D6093B9
:1009D000CC027093CD028093CE029093CF026091AF
:1009E000CC027091CD028091CE029091CF0220E096
:1009F00030E040E85BE30E94A50D6093CC02709369
:100A0000CD028093CE029093CF026091CC02709180
:100A1000CD028091CE029091CF020E94E60C70939D
:100A2000B2026093B1028091B1029091B2028093C0
:100A3000CB020F900F900F900F90CF91DF911F91ED
:100A40000F91FF90EF90DF90CF90BF90AF909F906D
:100A50000895482F8093AE026093AC026695669528
:100A600066956093C0028091BC029091BD0280386F
:100A700091057CF42091BC023091BD0280E890E0A9
:100A8000821B930B62E070E00E94270E460F40939A
:100A9000AE0284EA8093BC008091BC0087FFFCCF4B
:100AA0008091B0020E94CE0280E00E94CE0280912E
:100AB000C002806B0E94CE028091AE0282958F7040
:100AC00080610E94CE028091AE028F700E94CE02A1
:100AD00084E98093BC000895DF92EF92FF920F9318
:100AE0001F938091B302882311F400E001C00FEF3F
:100AF00010E084EAD82EB4E9EB2E612F660F660F62
:100B0000660F80E00E942905D092BC008091BC0055
:100B100087FFFCCF88E70E94CE0280E40E94CE02CD
:100B2000FF245BC0143071F1153040F41230C1F075
:100B30001330F8F4113009F049C008C01630A1F1A3
:100B4000163048F1173009F041C037C08091AA0231
:100B50009091AB0209970CF43CC0EE5AFC4F38C0A0
:100B60008091AA029091AB0241979CF1E259FA4F11
:100B70002FC08091AA029091AB02499754F1E053A3
:100B8000FD4F26C08091AA029091AB0281970CF193
:100B9000E652FB4F1DC08091AA029091AB0289974B
:100BA000C4F0EC5AFB4F14C08091AA029091AB02A2
:100BB000C1977CF0E059F94F0BC08091AA02909147
:100BC000AB02C99734F0E051FA4F02C0EC52FC4F2F
:100BD0000083802F0E94CE02F394EF2DF0E08091ED
:100BE000BC029091BD02E817F9070CF49BCFE0928C
:100BF000BC001F5F183009F080CF1F910F91FF904C
:100C0000EF90DF9008951F93182F84EA8093BC0023
:100C10008091BC0087FFFCCF8091B0020E94CE0281
:100C200080E40E94CE02812F0E94CE0284E980934C
:100C3000BC001F910895FF920F931F93082F80917E
:100C4000BF02823061F08330C9F08130F1F48091CD
:100C5000BC029091BD02861B602F082F16C08091A8
:100C6000BC029091BD02282F201B022F8091AA0266
:100C70009091AB02282F261B622F07C08091AA02F9
:100C80009091AB02801B062F682F262F2770162FFE
:100C90001695169516951430B1F1153040F41230B2
:100CA000D9F0133028F5113009F059C009C01630B9
:100CB00009F43FC0163090F1173009F050C044C01D
:100CC0008091AA029091AB0209970CF44DC0E02FDD
:100CD000F0E0EE5AFC4F47C08091AA029091AB021F
:100CE00041970CF441C0E02FF0E0E259FA4F3BC0CD
:100CF0008091AA029091AB024997B4F1E02FF0E005
:100D0000E053FD4F30C08091AA029091AB028197D1
:100D10005CF1E02FF0E0E652FB4F25C08091AA0283
:100D20009091AB02899704F1E02FF0E0EC5AFB4F71
:100D30001AC08091AA029091AB02C197ACF0E02F4B
:100D4000F0E0E059F94F0FC08091AA029091AB02F8
:100D5000C99754F0E02FF0E0E051FA4F04C0E02FC3
:100D6000F0E0EC52FC4FE0818091C602882351F004
:100D700081E090E002C0880F991F2A95E2F7FE2ECD
:100D8000F82A0AC081E090E002C0880F991F2A95D6
:100D9000E2F7F82EF094FE22EF1509F46FC0802FD1
:100DA0000E9429058F2D0E9403061430B1F11530E1
:100DB00040F41230D9F0133028F5113009F059C041
:100DC00009C0163009F43FC0163090F1173009F011
:100DD00050C044C08091AA029091AB0209970CF4D4
:100DE0004DC0E02FF0E0EE5AFC4F47C08091AA02C0
:100DF0009091AB0241970CF441C0E02FF0E0E25932
:100E0000FA4F3BC08091AA029091AB024997B4F18E
:100E1000E02FF0E0E053FD4F30C08091AA029091A6
:100E2000AB0281975CF1E02FF0E0E652FB4F25C06A
:100E30008091AA029091AB02899704F1E02FF0E033
:100E4000EC5AFB4F1AC08091AA029091AB02C19755
:100E5000ACF0E02FF0E0E059F94F0FC08091AA020A
:100E60009091AB02C99754F0E02FF0E0E051FA4FB7
:100E700004C0E02FF0E0EC52FC4FF0821F910F9184
:100E8000FF900895FF920F931F93082F8091BF0248
:100E9000823061F08330C9F08130F1F48091BC027E
:100EA0009091BD02861B602F082F16C08091BC0256
:100EB0009091BD02282F201B022F8091AA029091B1
:100EC000AB02282F261B622F07C08091AA029091A7
:100ED000AB02801B062F682F262F2770162F169522
:100EE000169516951430B1F1153040F41230D9F042
:100EF000133028F5113009F059C009C0163009F433
:100F00003FC0163090F1173009F050C044C08091B6
:100F1000AA029091AB0209970CF44DC0E02FF0E0CB
:100F2000EE5AFC4F47C08091AA029091AB024197C4
:100F30000CF441C0E02FF0E0E259FA4F3BC0809141
:100F4000AA029091AB024997B4F1E02FF0E0E05390
:100F5000FD4F30C08091AA029091AB0281975CF165
:100F6000E02FF0E0E652FB4F25C08091AA0290915D
:100F7000AB02899704F1E02FF0E0EC5AFB4F1AC066
:100F80008091AA029091AB02C197ACF0E02FF0E003
:100F9000E059F94F0FC08091AA029091AB02C99716
:100FA00054F0E02FF0E0E051FA4F04C0E02FF0E001
:100FB000EC52FC4FE0818091B302882351F081E034
:100FC00090E002C0880F991F2A95E2F7FE2EF82ABA
:100FD0000AC081E090E002C0880F991F2A95E2F7CD
:100FE000F82EF094FE22EF1509F46FC0802F0E94B6
:100FF00029058F2D0E9403061430B1F1153040F4FD
:101000001230D9F0133028F5113009F059C009C059
:10101000163009F43FC0163090F1173009F050C077
:1010200044C08091AA029091AB0209970CF44DC084
:10103000E02FF0E0EE5AFC4F47C08091AA02909159
:10104000AB0241970CF441C0E02FF0E0E259FA4FB7
:101050003BC08091AA029091AB024997B4F1E02F76
:10106000F0E0E053FD4F30C08091AA029091AB02B6
:1010700081975CF1E02FF0E0E652FB4F25C08091B4
:10108000AA029091AB02899704F1E02FF0E0EC5AAC
:10109000FB4F1AC08091AA029091AB02C197ACF0AD
:1010A000E02FF0E0E059F94F0FC08091AA02909133
:1010B000AB02C99754F0E02FF0E0E051FA4F04C0C2
:1010C000E02FF0E0EC52FC4FF0821F910F91FF9067
:1010D00008952F923F924F925F926F927F928F92DC
:1010E0009F92AF92BF92CF92DF92EF92FF920F93B7
:1010F0001F93DF93CF93CDB7DEB761970FB6F89408
:10110000DEBF0FBECDBFDC014C872D87EB860230E2
:1011100061F0033069F0013019F422E02F8302C03E
:1011200031E03F832224239407C082E08F8302C0F2
:1011300091E09F8392E0292E20E030E008C0FD017D
:10114000E20FF31F8081882329F02F5F3F4F26177E
:101150003707A8F31E8228873D0133244424FE016B
:101160003696FF87EE879E01295F3F4F398B288B8C
:1011700064C0F301908190525E010894A11CB11CDF
:1011800025E0929FF0011124E859FF4FD5019F35CA
:1011900010F08AEA01C084918D9331962E853F85A7
:1011A000A217B307A1F71E823AC0E114F10429F097
:1011B000882D6D2D0E941B0607C03B85332321F42B
:1011C000882D6D2D0E944207C3949394D394C2142A
:1011D00060F30F5F1F4F0830110579F0E984FA843E
:1011E000002E02C0F594E7940A94E2F781E0E82229
:1011F000FF24DD84D90CCC24D8CF5394439483941A
:101200009F81591620F4992400E010E0E7CF08945C
:10121000A11CB11CE889F989AE16BF0651F0F50191
:101220008081282F30E03A8729878C84840C5524CC
:10123000EACF33940894611C711C3885331608F486
:1012400098CF61960FB6F894DEBF0FBECDBFCF9199
:10125000DF911F910F91FF90EF90DF90CF90BF90A3
:10126000AF909F908F907F906F905F904F903F9046
:101270002F900895AF92BF92CF92DF92EF92FF929C
:101280000F931F93DF93CF9300D000D000D0CDB742
:10129000DEB76B015A01F22EE02EAA2797FDA0952A
:1012A000BA2FBC01CD018E010F5F1F4FA80126E0B0
:1012B00030E00E945D01C80166E070E0A601950182
:1012C0000F2D0E94690826960FB6F894DEBF0FBE58
:1012D000CDBFCF91DF911F910F91FF90EF90DF90E5
:1012E000CF90BF90AF900895EF92FF920F93DF934E
:1012F000CF9300D000D000D0CDB7DEB78091CB0225
:101300009091CB028F3F11F097FD04C08091CB02EA
:101310008F3F19F41092CB0254C01092BE029091EC
:10132000CB028091BE02282F30E040E050E09330A5
:1013300010F441E050E024233523232B09F441C06D
:1013400087E091E068E170E042E050E024E330E0C3
:1013500000E0EE240E94690885EC8093B50280913C
:10136000B50220E040EA5FE0CA010197F1F72F5F84
:101370002A3FD1F720E040EA5FE0CA010197F1F788
:101380002F5F2A3FD1F720E040EA5FE0CA010197D2
:10139000F1F72F5F2A3FD1F720E040EA5FE0CA0172
:1013A0000197F1F72F5F2A3FD1F78FE191E066E1D6
:1013B00070E042E050E024E330E000E0EE240E94E0
:1013C00069089091C5028091CB02981739F4109268
:1013D000B8021092C5021092CB020EC08091CB02CF
:1013E0008093C5029091B8028091CB02891720F0BA
:1013F0008091C5028093B8029091B8028091C40296
:10140000891708F048C085E391E067E170E042E0A9
:1014100050E024E330E000E0EE240E94690880E917
:1014200091E00E9441018CE491E065E170E042E0CE
:1014300050E024E330E00E94690880E991E00E94D6
:10144000410185EC8093B50281E691E068E170E0AE
:1014500042E050E024E330E00E9469088091C90234
:101460009091CA02069774F08091C1029091C202D5
:1014700001969093C2028093C1021092CA02109208
:10148000C90209C08091C9029091CA020196909345
:10149000CA028093C9029091AF028091B802981756
:1014A00020F48091B8028093AF028091AF0290E067
:1014B00062E470E046E150E020E000E00E943A097A
:1014C0006091AF0270E0882777FD8095982F7E01AC
:1014D0000894E11CF11CA70126E030E00E945D01A8
:1014E0008091B80290E062E470E04CE050E020E0CF
:1014F0000E943A096091B80270E0882777FD8095D4
:10150000982FA70126E030E00E945D018091C10282
:101510009091C2026CE570E046E150E020E00E944C
:101520003A096091C1027091C202882777FD8095C7
:10153000982FA70126E030E00E945D018CE291E047
:101540000E94410189E791E066E070E042E450E0EA
:101550002CE030E0EE240E9469088FE791E069E01A
:1015600070E042E450E026E130E00E9469082696EF
:101570000FB6F894DEBF0FBECDBFCF91DF910F91B4
:10158000FF90EF900895EF920F93DF93CF9300D0E9
:1015900000D000D0CDB7DEB788E891E066E170E01A
:1015A00042E050E022E030E000E0EE240E946908D2
:1015B0008EE991E06DE070E042E050E02CE030E038
:1015C0000E9469088BEA91E06AE070E042E050E036
:1015D00026E130E00E94690885EB91E06FE070E061
:1015E00042E050E020E230E00E9469088091C402AD
:1015F00090E063E670E040E250E020E00E943A09AB
:101600006091C40270E0882777FD8095982FAE0125
:101610004F5F5F4F26E030E00E945D0126960FB6D7
:10162000F894DEBF0FBECDBFCF91DF910F91EF9049
:101630000895EF920F9388E48093B8001092B90058
:101640008EEA0E94A50380E00E94A50380E40E9428
:10165000A50381E80E94A5038FEC0E94A50381EAFF
:101660000E94A50388EC0E94A50388EA0E94A503B6
:101670008091AA029091AB028034910511F48FE31E
:101680000FC08091AA029091AB02809741F08091A7
:10169000AA029091AB02409711F48FE001C08FE154
:1016A0000E94A50383ED0E94A50380E00E94A5038C
:1016B00085ED0E94A50380E80E94A50389ED0E94A4
:1016C000A50381EF0E94A5038AED0E94A50382E194
:1016D0000E94A5038091B402882311F082E101C029
:1016E00082E00E94A5038BED0E94A50380E40E9486
:1016F000A50380E20E94A50382E00E94A5038DE875
:101700000E94A50384E10E94A5038FEA0E94A5031D
:101710000E946C0580E060E00E94290584EC91E065
:1017200066E170E042E050E022E030E000E0EE24CC
:101730000E9469088AED91E066E170E042E050E0C5
:101740002CE030E00E94690880EF91E066E170E0F3
:1017500042E050E026E130E00E94690886E092E035
:1017600066E170E042E050E020E230E00E9469086B
:101770008CE192E066E170E042E050E02AE230E085
:101780000E94690882E392E065E170E042E050E087
:1017900024E330E00E94690830E040EA5FE01EC0C8
:1017A000CA010197F1F72F5F2A3FD1F720E0CA0164
:1017B0000197F1F72F5F2A3FD1F720E0CA01019787
:1017C000F1F72F5F2A3FD1F720E0CA010197F1F727
:1017D0002F5F2A3FD1F73F5F333011F020E0E0CF99
:1017E0000E946C050F91EF900895BF92CF92DF9207
:1017F000EF92FF920F931F93CF93DF9314BE14BE0B
:1018000088E10FB6F89480936000109260000FBEDC
:101810001092C30281E28093C40288E78093B002F1
:1018200080E490E09093AB028093AA0280E890E07D
:101830009093BD028093BC0281E08093B402109229
:10184000BF021092B3028FEF8093C60281E090E056
:101850009093B7028093B6021092BB021092BA0224
:101860000E94190B11E0C0EADFE044E9B42E38E42D
:10187000F32ECC24CA9424E4D22E0E941304109395
:10188000AD028091AD02882309F442C08091B90273
:10189000882319F00E947409F0CF1092C3021093AC
:1018A000B90287E492E063E170E042E050E02CE0AE
:1018B00030E000E0EE240E94690820E0CE010197AC
:1018C000F1F72F5F2A3FD1F720E0CE010197F1F722
:1018D0002F5F2A3FD1F720E0CE010197F1F72F5F6C
:1018E0002A3FD1F720E0CE010197F1F72F5F2A3F81
:1018F000D1F78AE592E067E170E042E050E02CE049
:1019000030E000E0EE240E9469080E94C30AB5CFCF
:101910008091C302882319F00E940303AECF0E9476
:101920006C051093C3021092B90281E792E062E164
:1019300070E042E050E02CE030E000E0EE240E9455
:10194000690883E892E066E170E042E050E026E159
:1019500030E00E94690830E01EC0CE010197F1F727
:101960002F5F2A3FD1F720E0CE010197F1F72F5FDB
:101970002A3FD1F720E0CE010197F1F72F5F2A3FF0
:10198000D1F720E0CE010197F1F72F5F2A3FD1F781
:101990003F5F323011F020E0E0CF0E946C058FEA0B
:1019A0000E94A503B092BC001092B900F092B8005A
:1019B000F092BA00C092BD00D092BC0020E0CE01EF
:1019C0000197F1F72F5F2436D1F757CF04D06894F1
:1019D000B111B5C0089598D088F09F5790F0B92FF5
:1019E0009927B751A0F0D1F0660F771F881F991F74
:1019F0001AF0BA95C9F712C0B13081F09FD0B1E0AA
:101A000008959CC0672F782F8827B85F39F0B93FB9
:101A1000CCF3869577956795B395D9F73EF4909575
:101A20008095709561957F4F8F4F9F4F0895E894F3
:101A300009C097FB3EF490958095709561957F4F16
:101A40008F4F9F4F9923A9F0F92F96E9BB279395C4
:101A5000F695879577956795B795F111F8CFFAF4D4
:101A6000BB0F11F460FF1BC06F5F7F4F8F4F9F4F05
:101A700016C0882311F096E911C0772321F09EE863
:101A8000872F762F05C0662371F096E8862F70E0C9
:101A900060E02AF09A95660F771F881FDAF7880FA3
:101AA0009695879597F9089597F99F6780E870E074
:101AB00060E008959FEF80EC089500240A941616C4
:101AC000170618060906089500240A94121613062C
:101AD000140605060895092E0394000C11F48823BA
:101AE00052F0BB0F40F4BF2B11F460FF04C06F5FD6
:101AF0007F4F8F4F9F4F089557FD9058440F551FAC
:101B000059F05F3F71F04795880F97FB991F61F07F
:101B10009F3F79F087950895121613061406551FF6
:101B2000F2CF4695F1DF08C0161617061806991F62
:101B3000F1CF86957105610508940895E894BB2757
:101B400066277727CB0197F908950BD0C4CFB5DF6F
:101B500028F0BADF18F0952309F0A6CFABCF1124F7
:101B6000EECFCADFA0F3959FD1F3950F50E0551F3C
:101B7000629FF001729FBB27F00DB11D639FAA27E2
:101B8000F00DB11DAA1F649F6627B00DA11D661F31
:101B9000829F2227B00DA11D621F739FB00DA11D52
:101BA000621F839FA00D611D221F749F3327A00D0C
:101BB000611D231F849F600D211D822F762F6A2FA8
:101BC00011249F5750408AF0E1F088234AF0EE0F2D
:101BD000FF1FBB1F661F771F881F91505040A9F73A
:101BE0009E3F510570F060CFAACF5F3FECF3983E67
:101BF000DCF3869577956795B795F795E7959F5FA1
:101C0000C1F7FE2B880F911D9695879597F908953A
:101C1000629FD001739FF001829FE00DF11D649FD0
:101C2000E00DF11D929FF00D839FF00D749FF00D5C
:101C3000659FF00D9927729FB00DE11DF91F639FFD
:101C4000B00DE11DF91FBD01CF011124089597FBCF
:101C5000092E07260AD077FD04D02ED006D000200A
:101C60001AF4709561957F4F0895F6F790958195D8
:101C70009F4F0895A1E21A2EAA1BBB1BFD010DC0A8
:101C8000AA1FBB1FEE1FFF1FA217B307E407F5072C
:101C900020F0A21BB30BE40BF50B661F771F881F08
:101CA000991F1A9469F760957095809590959B019E
:101CB000AC01BD01CF010895AA1BBB1B51E107C0B8
:101CC000AA1FBB1FA617B70710F0A61BB70B881FCC
:101CD000991F5A95A9F780959095BC01CD0108955B
:041CE000F894FFCFA6
:101CE4000020003000000050726573733D302C20DA
:101CF40070756D70206973204F6E212121200020A2
:101D040020202020202020202020202020202020CF
:101D140020202020005072657373757265206973EA
:101D24002020204D61782020202020004973207439
:101D34006865204C696E6520626C6F636B65643FF7
:101D440000202020202020202020202020202020AF
:101D540020202020202020200020202020200020BF
:101D64002020202020202000487837313062202B8A
:101D7400204D5058353031304450202020005072CE
:101D8400657373206E6F7720202000507265737323
:101D9400206D617800576174657250756D70206DA7
:101DA40061783D004F6C65645F496E69745F4F4BA9
:101DB4003132335F3132333435002D2D2D2D2D2D1D
:101DC4002D2D2D2D2D2D2D2D2D2D2D2D2D2D2D006C
:101DD4004153444647484A4B4C5A584356424E4D49
:101DE4002C2E2F3132002E2E2E2E2E2E2E2E2E2E37
:101DF4002E2E2E2E2E2E2E2E2E2E2E005A5843569A
:101E0400424E4D3C3C3C3E3E3E3F3F3F3F7B7B7B16
:101E14007D002D2D2D2D4C494E453D3D3D365F5FBA
:101E24005F5F5F5F2D2D004E616E6F2061732069CF
:101E34003263204D617374657200202020202020BD
:101E4400202020202020202020202020202020208E
:101E5400004E616E6F2061732069326320536C61A0
:101E6400766500537769746368696E6720446973A3
:101E7400706C6179204F666600200000000000004D
:0C1E840000000000000000000000400012
:00000001FF
